:100000008C289200220884000930930003100D20F0
:10001000920C930B072803140D2884139F1D1C2892
:10002000000820041F1D20068000841700082004FB
:10003000031C20068000272800082004031C20063B
:100040001F192006800084172009800527281F0D0E
:1000500006398C0030208D008C0A302000004A28A0
:1000600000308A000C0882070134753403341534DB
:1000700000343C340C34D9348F018E00FF308E07AD
:10008000031C8F07031C872803308D00DF304A20B4
:100090003E288D01E83E8C008D09FC30031C53285E
:1000A0008C07031850288C0764008D0F50280C18FB
:1000B00059288C1C5D2800005D28080093019200DF
:1000C0001C308E006F308F0071200F30831681043A
:1000D0008312FF3063008C07031C8D0703186A2806
:1000E0008728103094008D018C01930C920C031C16
:1000F0007F280E088C070F0803180F0F8D078D0C33
:100100008C0C910C900C940B752810088728831385
:100110000313831264000800831685010F308600E4
:10012000831201305E20C030860005303C20060876
:10013000A400F03086000F302405A50064002508D7
:100140000E3C031DBD280530A2000430A00006307F
:100150009F00FE300120013001202030012020309E
:100160000120203001204E3001206F3001207230FC
:1001700001207430012068300120640025080C3C07
:10018000031DE6280530A2000430A00006309F00C1
:10019000FE300120013001202030012020300120DC
:1001A000203001204E3001206F30012072300120BC
:1001B00074300120683001202D30012045300120AD
:1001C0006130012073300120743001206400250863
:1001D0000D3C031D03290530A2000430A0000630A9
:1001E0009F00FE300120013001202030012020300E
:1001F0000120203001204530012061300120733082
:1002000001207430012064002508093C031D2C29BD
:100210000530A2000430A00006309F00FE3001200F
:100220000130012020300120203001202030012029
:10023000533001206F3001207530012074300120CF
:10024000683001202D30012045300120613001202F
:100250007330012074300120640025080B3C031D1D
:100260004B290530A2000430A00006309F00FE306C
:1002700001200130012020300120203001202030D9
:100280000120533001206F3001207530012074307F
:1002900001206830012064002508033C031D7429F7
:1002A0000530A2000430A00006309F00FE3001207F
:1002B0000130012020300120203001202030012099
:1002C000533001206F30012075300120743001203F
:1002D000683001202D300120573001206530012089
:1002E000733001207430012064002508073C031D91
:1002F00091290530A2000430A00006309F00FE3096
:100300000120013001202030012020300120203048
:1003100001205730012065300120733001207430F6
:10032000012064002508093C031DBA290530A200FC
:100330000430A00006309F00FE3001200130012073
:100340002030012020300120203001204E300120BB
:100350006F3001207230012074300120683001209C
:100360002D300120573001206530012073300120ED
:0A0370007430012091286300BB29BE
:02400E00FD3F74
:00000001FF
